:10000000020F719404E50C9400223202120B90014D
:1000100000E004F0785AE66001169000FBE0600210
:0700200014F02202000A3275
:03002B0002107C44
:10003300020026BB010689828A83F0225002F7223E
:10004300BBFE01F322EF8DF0A4A8F0CF8CF0A4281F
:10005300CE8DF0A42EFE22BC000BBE0029EF8DF046
:1000630084FFADF022E4CCF875F008EF2FFFEE33F8
:10007300FEEC33FCEE9DEC984005FCEE9DFE0FD5A7
:10008300F0E9E4CEFD22EDF8F5F0EE8420D21CFE7B
:10009300ADF075F008EF2FFFED33FD4007985006E4
:1000A300D5F0F222C398FD0FD5F0EA22C2D5EC3089
:1000B300E709B2D5E4C39DFDE49CFCEE30E715B23D
:1000C300D5E4C39FFFE49EFE12005AC3E49DFDE402
:1000D3009CFC800312005A30D507C3E49FFFE49EC3
:1000E300FE22C5F0F8A3E028F0C5F0F8E5821582FA
:1000F30070021583E038F022E88FF0A4CC8BF0A4D3
:100103002CFCE98EF0A42CFC8AF0EDA42CFCEA8EE6
:10011300F0A4CDA8F08BF0A42DCC3825F0FDE98F09
:10012300F0A42CCD35F0FCEB8EF0A4FEA9F0EB8F00
:10013300F0A4CFC5F02ECD39FEE43CFCEAA42DCECD
:1001430035F0FDE43CFC2275F008758200EF2FFFCB
:10015300EE33FECD33CDCC33CCC58233C5829BED9C
:100163009AEC99E58298400CF582EE9BFEED9AFDA0
:10017300EC99FC0FD5F0D6E4CEFBE4CDFAE4CCF950
:10018300A88222B800C1B90059BA002DEC8BF084C3
:10019300CFCECDFCE5F0CBF97818EF2FFFEE33FE91
:1001A300ED33FDEC33FCEB33FB10D703994004EB49
:1001B30099FB0FD8E5E4F9FA227818EF2FFFEE3315
:1001C300FEED33FDEC33FCC933C910D7059BE99A27
:1001D3004007EC9BFCE99AF90FD8E0E4C9FAE4CCB8
:1001E300FB2275F010EF2FFFEE33FEED33FDCC3322
:1001F300CCC833C810D7079BEC9AE899400AED9B0B
:10020300FDEC9AFCE899F80FD5F0DAE4CDFBE4CCE9
:10021300FAE4C8F922E8600FECC313FCED13FDEE1A
:1002230013FEEF13FFD8F122A42582F582E5F03502
:1002330083F58322E493FB740193FA740293F92206
:10024300D083D082F8E4937012740193700DA3A34A
:1002530093F8740193F5828883E47374029368605E
:10026300EFA3A3A380DFEC8EF0A4CCC5F0CCCDF834
:10027300EFA4CEC5F02DFDE43CFCE8A42EC8C5F0E8
:100283003DFDE43CFCEFA4FFE5F028FEE43DFDE486
:100293003CFC228F358C368D37E4F543F544F5412C
:1002A300F542F538E538C3953540030203809000E5
:1002B300B5E0FF6538701CE5192FFFE412080CFC4C
:1002C300A3E0FD1207F7FEA3E0C39DF540EE9CF506
:1002D3003F80641207E31208031208D08F3C8E3B61
:1002E3008D3A8C39E5192538FFE41207EE1208E63A
:1002F300AF3CAE3B1201868E3D8F3E1207E31208E0
:10030300031208DB953EFFEE953DAB07FAE4F9F8DF
:10031300AF3CAE3BAD3AAC391201868E3D8F3E9079
:1003230000B5E02519FFE41207EEFEA3E0C3953EF6
:10033300F540EE953DF53FC3E53F6480948050055D
:10034300E4F53FF540D3E5409542E53F9541401440
:10035300854546854143854244853845853F4185EA
:1003630040428014D3E5409544E53F9543400985D9
:100373003846853F4385404405380202A7E54225B8
:1003830044FFE5413543FEC3EF9537EE95365005FF
:100393007EFF7FFF22E536C313FEE53713FFC3E578
:1003A300429FF540E5419EF53FFEAF407C007D0A4C
:1003B3001200481208B9EDD3941F40027D1FEDAC23
:1003C30036AD37120875CEC313CE13D8F9F53E8E6A
:1003D3003D2542F542E53D3541F541E53E2544F5F0
:1003E30044E53D3543F543E544AE437807C333CE97
:1003F30033CED8F9FF1208B9900124E07002A3E0CC
:100403007005120892800D1208C3CEC313CE13D801
:10041300F912084B1208F0CEC313CE13D8F9FD908E
:1004230000D0E545F075F040A485F047F548E54573
:100433001208A25002AD07E545120821C333CE339B
:10044300CED8F9120833AD07AC06E545700AE53599
:1004530014B54604C206801BE53514B54508E546C8
:100463007004D206800DE545C395465004D206803C
:1004730002C20630060CED2548F548EC3547F54732
:100483008022E54845477011E53575F040A4AEF08C
:1004930024FFF548EE34FFF547C3E5489DF548E5ED
:1004A300479CF547AE47AF4822E4F532F5F875FBB4
:1004B3003FD20153D57F43D501E5F854F84407F5FE
:1004C300F853F8BF75F90F75FA329081037440F051
:1004D300E4F5E8F5C0908030F090FC00E04440F093
:1004E300E58654F04407F586E4F5161213EA75A180
:1004F300A575D58075D67FE532601F908030E054B6
:100503007FF0E054FE4401F0C2AF438702000000D5
:10051300E04480F0E054FEF0D2AF900100E0FFC36E
:1005230094054003020620E5FB60CCEF600214F063
:10053300E4FD7E007401A805088005C333CE33CEE5
:10054300D8F9FFACFBECFBEF5B70030205F0A805E9
:100553007401088002C333D8FCF5FBED700885E213
:100563003385E1348035BD010885E43385E3348088
:100573002ABD020885E63385E534801FBD0308855F
:10058300D93385E7348014BD040885DB3385DA3439
:100593008009BD050685DD3385DC34E532702CE545
:1005A3003424F7FFE53334FFFEE5162DFC1209D69C
:1005B300EEF0A3EFF0E5342409FFE43533FEEC124B
:1005C3000A08F583EEF0A3EFF08022E5162DFF1263
:1005D30009D6E0FAA3E0C39534EA9533503FEF120E
:1005E3000A08120962D39534EE953340300DED6459
:1005F300066003020535E5162406120985500874C2
:10060300062516F516800DE4F516E53270067532EB
:100613000143F8201213EA75A1A50204FAE4F5F8E0
:1006230075FB3FE58654F0440DF5861209C99080A9
:1006330030E04440F053D57F43D5017F017E001263
:10064300143075D580E4F5D6F5161211BD120A01E2
:10065300C20175E8E322C205751908200307D20316
:100663007F0412124C7D4A7C007F04120296EFF441
:100673007002EEF46002C204900123E0F960030209
:100683000763900122E06003020733EFF47002EE88
:10069300F4600B7401F09000FF04F00207B38519B6
:1006A3003212094340030207B3120924E532120947
:1006B30018E0FAA3E0FBD39DEA9CE5324007120958
:1006C30026C3EB8014120918E0FCA3E0FDE5321207
:1006D30009A7F583E0FAA3E0C39DF534EA9CF5335B
:1006E300D3E5349408E5339400502174162532126F
:1006F300093BE07036120924E532120918ECF0A325
:10070300EDF0120924E5321209F7800E120924E5EF
:100713003225E02402F582E43400F583ECF0A3ED06
:10072300F07416253212093B7432F005320206A426
:10073300EFF47002EEF4600D9000FFE07072900130
:100743002304F0806BE4900122F0851932120943EF
:10075300505E7416253212093B7432F0053280ED77
:10076300E96401704B900122E06011EFF47002EE36
:10077300F4703DF09000FF7402F08034EFF47002E7
:10078300EEF470269000FFE07026900123F0A3F0B2
:10079300A31209B185193212094350147416253274
:1007A30012093B7432F0053280ED9001227401F09E
:1007B300900123E0B40112EFF47002EEF4600D90A7
:1007C30000FCEEF0A3EFF080031209B29000FCE00E
:1007D300F47003A3E0F4600475180222E4F5182210
:1007E3009000B5E0AD197C002DFFEC33FEEF25E062
:1007F300FFEE33FE741A2FF58274003EF583E02278
:10080300FAA3E0FBED2538FFEC33FEEF25E0FFEE26
:1008130033FE74B62FF58274003EF583E022901503
:100823007C93FCFFEDC39FFFE49400FEEF78052269
:10083300FFECFDC374809DFDE49400FC0200AF75E2
:10084300F00290001A02022BFFC3EB9FFFEA9E9077
:100853000124F0A3EFF0EDFF900124E48FF00200F8
:10086300E5E5009000B675F00212022BE0FEA3E06E
:10087300FF22FFC374209FFFE49400FE120048EFA1
:10088300780622C3EB9FEE6480F8EA64809822ED39
:1008930075F004A4FF900124E5F0F0A3EFF022909B
:1008A300157C93FFEDC39F22E500C313FEE5001300
:1008B300FFC3E5009F22AC41AD4212005AAD0722AF
:1008C300900124E0FAA3E0FBAE02780222FEA3E04B
:1008D300FFAD03AC02020269FEA3E02BFFEE3AFE7A
:1008E300C3EF22FEA3E0FBAA06E4F9F82290012459
:1008F300E0FEA3E0780222AC00AD0012005AAD077F
:1009030022E53225E024B6F582E43400F583E0FEE7
:10091300A3E0FFE53225E02402F582E43400F58309
:1009230022E53225E024B6F582E43400F583E0FCC9
:10093300A3E0FD2274162532F582E43401F5832207
:10094300E5192404FDE433FCC3E5329DEC6480F82F
:1009530074809822E53225E024D1F582E43400F551
:1009630083E0FEA3E02274012532F582E43401F52D
:100973008322E53275F00AA42432F582E43400F5CB
:100983008322FFE433C3FE7859E6FDEF9D7480F8BC
:100993006E982225E0241AF582E43400F583EEF004
:1009A300A3EFF02225E024B6F582E4340022F074AC
:1009B300FF9000FCF0A3F022E53290158093FF78BE
:1009C3005BE6FEEF5E2275F90A75F84090810374C9
:1009D30057F02225E02428F582E43401F5832278B8
:1009E30059E62401FFE433FEC32225E024D1F58236
:1009F300E434002225E0241AF582E4340022900036
:100A0300FB7405F02225E02440F582E4340122E45E
:100A1300F530F52FF52EF52DF53175E8E39080309F
:100A2300E04440F075A081E4F5A375A24B75A1A540
:100A3300D2AF120FFD90801A7402F0C2B212128D5F
:100A4300E48F308E2FF52EF52DAD2EAC2D780812B8
:100A530002188F1385301485140F8513105389FCE6
:100A6300758CFB758A1BC28CD2A9C2B91210FA907D
:100A730000FCE0FEA3E0FFF47002EEF4601B754996
:100A830001E4F54B75310174592FF58274143EF569
:100A930083E493F54A240FF54A9000FEE0FF60518A
:100AA300754901E4F54BEF1202430AC9010ACE026C
:100AB3000AD3040AD8080ADD100AE2200AE7400A2A
:100AC300EC8000000AF1754A058026754A0C8021E6
:100AD300754A0A801C754A0B8017754A098012757E
:100AE3004A07800D754A038008754A018003E4F5BF
:100AF300499000FCE0B4FF0EA3E0B4FF099000FEB0
:100B0300E07003754B01E54964016003020A6FF568
:100B130049D28C854A11020A6FE50914602C1460CE
:100B230048147003020BFC24036003020C18D2B2B6
:100B3300050DE50D7002050CC31200035003020CF2
:100B430018E4F50CF50D75090122C2B2050DE50D8A
:100B53007002050CC39478E50C94005003020C1842
:100B6300E4F50CF50D75090222E512700B751201FF
:100B7300740F250AF8E6F50B050DE50D7002050C5B
:100B8300E50B30E726D3E50D940CE50C94005004F7
:100B9300D2B28044C3E50D940DE50C94004039C2F4
:100BA300B2E50D6410450C702F8021D3E50D1200C2
:100BB300035004D2B28021C3E50D9405E50C9400E3
:100BC3004016C2B2E50D6410450C700CF50CF50D22
:100BD300E50B25E0F50B050EE50E64087037F50E01
:100BE300F512050AE50A6403702BF50AE54BB40117
:100BF3000475090322E4F50922050DE50D700205CC
:100C03000CD31200035003D2B222C2B2E4F50CF5A6
:100C13000DF509C28C22E4F532120916E0FCA3E0BB
:100C2300FD120CFE8F33E532120926120CFE8F34AF
:100C3300E53464026008E53464036002C204E5330A
:100C43007030E534701B1209BB700E120937E06077
:100C530003020CE1EF4EF680001209377402F080B4
:100C63007D1209BB6069120937E07072EFF45EF61A
:100C73008015E534700C120904EEF0A3EFF0E4FDE7
:100C83008057785BE66011E5321209F712090FEE1F
:100C9300F0A3EFF07D028041120916E0FEA3E0FF0E
:100CA300E5321209267B1E7A00121364EF602012CC
:100CB3000937E07029120904EEF0A3EFF0E53212D0
:100CC30009A7120962FFE5321209967D02800A1212
:100CD3000904EEF0A3EFF0AD34AF3212144605323F
:100CE300E532C394085003020C1C785BE69000FEC7
:100CF300F0600475180122E4F51822E5329015809E
:100D030093785B5624FF92057B1E7A00AF32121153
:100D13005E229000B4E07015C200900100F0F51659
:100D23001211BD9000B47402F0751532229000B414
:100D3300E064026003020DED200003020DEDC2002A
:100D43001515E5156003020DED785AF6F532120913
:100D5300E2E5329FEE1209504003020DE9E4FFE59C
:100D6300321209ED12092FE53212097775F002EFFD
:100D730012022BECF0A3EDF00FBF05E37401253253
:100D830012096DE4F0E532785966605A120957FF8B
:100D9300E532120996120957FFE532120918EEF0EF
:100DA300A3EFF0E532C39408502DE53225E025E0AA
:100DB300245AF582E43415F583E493FE740193FF1A
:100DC300E53225E024EBF582E4340012099F7D022D
:100DD300AF32121446800A7416253212093B74325C
:100DE300F00532020D51784C760122908109E054CE
:100DF300E06004E044E0F0E5FB30E00975FB0185C9
:100E0300E22185E122E5FB30E10975FB0285E4235C
:100E130085E324E5FB30E20975FB0485E62585E5DA
:100E230026E5FB30E30975FB0885D92785E728E527
:100E3300FB30E40975FB1085DB2985DA2AE5FB30F5
:100E4300E50975FB2085DD2B85DC2CE4FFEF25E030
:100E53002421F8E6FC08E6FDE5162F1209EDF583DB
:100E6300ECF0A3EDF0EFFDE5162DFDE433FC78592E
:100E7300E66D7001EC60040FBF06D2E5162406FF91
:100E8300E433D31209894007D200E4F516800674CF
:100E9300062516F5161211BD900100E0600214F04C
:100EA300900127E0FF900126E0FE6F6006A3EEF0BD
:100EB30075A1A522E4F5321209E2E5329FEE12098B
:100EC300504003020F70120969E004F0120969E04F
:100ED300C394054005120969E4F0C2ADE532120975
:100EE30059FF120975C083C082120969E0D082D00C
:100EF3008375F00212022BEEF0A3EFF0D2ADE4F50E
:100F030033F534F535F53674FFF537F538E4FF126C
:100F1300097575F002EF12022BE0FCA3E0FD253406
:100F2300F534EC3533F533D3ED9536EC9535400494
:100F33008C358D36C3ED9538EC953750048C378D51
:100F4300380FBF05CAC3E5349536FFE5339535FE43
:100F5300C3EF9538FFEE9537FE7C007D0312005AF0
:100F6300E5321209A712099F0532020EBA22787FD1
:100F7300E4F6D8FD75815D020FB8020A12E493A36B
:100F8300F8E493A34003F68001F208DFF48029E438
:100F930093A3F85407240CC8C333C4540F4420C884
:100FA300834004F456800146F6DFE4800B0102041B
:100FB3000810204080901392E47E019360BCA3FF4D
:100FC300543F30E509541FFEE493A360010ECF5450
:100FD300C025E060A840B8E493A3FAE493A3F8E43F
:100FE30093A3C8C582C8CAC583CAF0A3C8C582C8AB
:100FF300CAC583CADFE9DEE780BE7859760CE4FF11
:10100300FEEEC39408EE501125E025E02458F58246
:10101300E43415F5837401800390157093FDAC07D8
:101023000F744D2CF8A6050EBE0CD6908030E0440C
:1010330040F075D580E4F5D6D2AD1213351209C947
:10104300D2ADC200E49000FEF0785BF6F518120A08
:1010530001D202C201C203E4900123F090012212E3
:1010630009B1E4900124F0A3F0784CF69000B4F0B9
:10107300900127F0900126F022C0E0C0F0C083C0A9
:1010830082C0D075D000C000C001C002C003C0043C
:10109300C005C006C007E5D530E03743D5013001B0
:1010A30008900100E004F080331212FFE51D451C97
:1010B3006008E51D151D7002151C051EE51EC39471
:1010C300804006751E0012000EE508C394FA500214
:1010D3000508200107E5FB6003120DEED007D006DB
:1010E300D005D004D003D002D001D000D0D0D0821C
:1010F300D083D0F0D0E032784CE614600604705A06
:10110300020D15300042C200900127E00490012631
:10111300F0120EB7D204E51864026003120C19E54D
:101123001864016003120659300408300205E5878C
:1011330030E203120A019000FBE0700C3002097FD9
:1011430001FE1214151204AC900100E0C394054093
:1011530009E4F5F875FB3F120FFD228A358B36A99A
:1011630007E9120842E0FEA3E0C39DFFEE9CAB0734
:10117300FAE99000EB12086930050B7C007D091237
:1011830000480D1200AF12088640037F0022D3EB04
:101193009536E53512088A40037F0122C3EA64804D
:1011A300948040037F0222C3E49536FFE49535FE25
:1011B3001208867F0440027F0322E4FEEEC39406F6
:1011C3005042EEFDE5162DFDE433FC7859E6FBC3F2
:1011D300ED9B7480F86C98401AAF067D0E1212C70F
:1011E300EE04FCECC39406501BAF04E4FD1212C7DB
:1011F3000C80F0AF06E5162E244DF8E604FD12121E
:10120300C70E80B843F88022C0E0C0F0C083C0821C
:10121300C0D075D000C000C001C002C003C004C06C
:1012230005C006C007758CFB758A1B120B1CD00703
:10123300D006D005D004D003D002D001D000D0D046
:10124300D082D083D0F0D0E032A90774FFF535F512
:1012530036AF19E4FEE92519FDE433FCEFC39DEC39
:101263006480F8748098502175F002EF120845E00D
:10127300FCA3E0FDC39536EC953550099000B5EE1F
:10128300F08C358D360F0E80CC2290FC017480F0EB
:10129300E490FC06F090FC05F090FC017481F0A34F
:1012A300E0FFE48F35F534F533F532AE34AD33ACCE
:1012B300321213C21213BE1213BEF532E490FC01B4
:1012C300F0AC3222EF14601614601914601C146021
:1012D3001F14602224057023ED4440F5FC22ED44E5
:1012E30040F5FD22ED4440F5FE22ED4440F5FF229A
:1012F300ED4440F5F122ED4440F5F222900000E088
:1013030004F0E0C394044029E4F0FF7859E6FEEFCB
:10131300C39E501574162F12093BE0600974162FF3
:1013230012093BE014F00F80E29000FFE06002142A
:10133300F02290801D7404F0E4FF7859E6FEEFC3B9
:101343009E501D744D2FF8E675F003A4248DF5828D
:10135300E43415F58312023774041200360F80DA71
:1013630022C3EF9DFFEE9CFED3EF9BEA6480F8EE71
:101373006480985017C3E49BFDE49AFCC3EF9DEC93
:101383006480F8EE64809840037F01227F0022018D
:101393004900014A00014B00011E00010900020C33
:1013A3000000030F000000010A00010E00010B0002
:1013B3000112004100000001150000F532FCE4FBBE
:1013C3007A01F9F81200FB8F358E348D338C32900D
:1013D300FC02E0FFE5354FFFE534FEE533FDE53282
:1013E3008F358E348D3322E4F535E5162535120914
:1013F30085500BE5162535244DF8E6048001E4FD00
:10140300AF351212C70535E535C3940640DC43F802
:1014130080228F828E83E5821582AE8370021583CC
:101423004E60097F147E0012143080EA22EF1FAA57
:101433000670011E4A600BE4FDEDC3944750EE0DA8
:1014430080F722ED90158893FE74162FF582E4340D
:1014530001F583EEF02200010203040506070809E3
:101463000A0B0C0D0E0F1011121213141516171868
:10147300191A1B1C1D1E1F20212223242525262764
:1014830028292A2B2C2D2E2F303132333435363761
:101493003838393A3B3C3D3E3F4041424344454660
:1014A3004748494A4A4B4C4D4E4F5051525354555D
:1014B300565758595A5B5C5D5D5E5F606162636459
:1014C30065666768696A6B6C6D6E6F707071727355
:1014D3007475767778797A7B7C7D7E7F8081828252
:1014E300838485868788898A8B8C8D8E8F90919251
:1014F30093949595969798999A9B9C9D9E9FA0A14E
:10150300A2A3A4A5A6A7A8A8A9AAABACADAEAFB049
:10151300B1B2B3B4B5B6B7B8B9BABABBBCBDBEBF46
:10152300C0C1C2C3C4C5C6C7C8C9CACBCCCDCDCE42
:10153300CFD0D1D2D3D4D5D6D7D8D9DADBDCDDDE40
:10154300DFE0E0E1E2E3E4E5E6E7E8E9EAEBECED3E
:10155300EEEFEFF0F0000000640001006400020011
:10156300C80003005A0004005A0005006400060086
:10157300FA0007012C080B0A094628284601020431
:1015830008102040800264501E1E0180190180183B
:1015930001800701800601800501800401800301A9
:1015A300800201800101800001801C01801B0180F9
:0115B3001A1D
:00000001FF
